:020000000F28C7
:080008000B110900F6000030A5
:100010008A000F30760703188A0A7608820783124F
:100020000313B401B501E030B6000130B700B800E9
:10003000B901BA01BB01BC01BD01D0018312031398
:10004000D1010130D200D301E901E03083168500EF
:10005000F0308600403081008B01BA246830831272
:100060000313DC003123F1005508F0007108A600ED
:100070007008A7003108A9003008A8007030DC0023
:100080003123F1005508F0007108AA007008AB0098
:100090003108AD003008AC007830DC003123F100CD
:1000A0005508F0007108B2007008B300CD010130AE
:1000B000CC00CF01CE014030E1003225CD0102302D
:1000C000CC00CF01CE015030E1003225FA30FE00E5
:1000D0006F25831203135308F0005208031D732881
:1000E00070020319A228CD010130CC00CF01CE014E
:1000F000E1013225CD010230CC00CF01CE0110301C
:10010000E10032250130D8000330D9002708C100B2
:100110002608C0002908C3002808C2007522023042
:1001200083120313D8000330D9002B08C1002A081A
:10013000C0002D08C3002C08C200752283120313CF
:10014000D201D30132082602F1003308031C013E1C
:100150002702F0007108E03EF1000318F00A0130B8
:10016000F0077108F9007008FA000830FB00FC0184
:100170006024F0007808831203132807F1000318A5
:10018000F00A2908F0077108BE007008BF00C630E9
:10019000D700EB2183122A08F9002B08FA00083057
:1001A000FB00FC016024F0007808831203132C0785
:1001B000F1000318F00A2D08F0077108BE0070085E
:1001C000BF00C030D700EB21C7308312D600D92141
:1001D000E800FF306802031DF0283F30E700F728F1
:1001E000681FF5282A30E700F7282130E7000130A2
:1001F000C4000C30C6006708DA001723C130831230
:100200000313D600D921E800FF306802031D0B2933
:100210003F30E7001229681F10292A30E700122911
:100220002130E7000230C4000C30C6006708DA0055
:100230001723831203130608F000F00CF00CF00CE7
:10024000700C0F39F0007008073C031D5129FD2484
:1002500083120313CD010130CC00CF01CE01203039
:10026000E1003225BB08031D3E29BA08031D3E29C3
:100270000830E9000130BA00BB014129E901BA01A7
:10028000BB010130C4006908C6002330DA0017231F
:10029000FA30FE006F25013083120313D200D30120
:1002A000D52970080B3C031D8429831203132B08E6
:1002B000AF002A08AE002D08B1002C08B0000230B3
:1002C000B800B9013308D1003208D000B201B3013F
:1002D000B601B701C030E5007030E6008526831214
:1002E00003132F08AB002E08AA003108AD00300818
:1002F000AC005108B3005008B200E030B600013045
:10030000B700D200D301D52970080C3C031DAC29DD
:10031000FD2483120313CD010130CC00CF01CE01A7
:100320003030E10032252708AF002608AE00B001CA
:10033000B1010130B400B5010130B800B901BA0112
:10034000BB01C630E5007830E60085260130831217
:100350000313D200D301D52970080D3C031DD02909
:10036000831203132708AF002608AE002908B10046
:100370002808B0000130B800B901C630E500683087
:10038000E6008526831203132F08A7002E08A60077
:100390003108A9003008A8000130D200D301D529C6
:1003A00070080E3C031DD529D5293230FE006F257B
:1003B00069288B25831203135608E200AE254C26CC
:1003C000EA001726E030831603138500F03086001C
:1003D00083126A08080083160313A001A1010030EC
:1003E00021020130031CFC290030031DFC290430CC
:1003F0002002013003180301003C03192B2A831249
:100400003E08F8003F08F7001030FA00F901822496
:10041000F1007D08F100831603132108F200200883
:100420006C3E8400710883138000831203133E081E
:10043000F8003F08F7001030FA00F9019E24F1009F
:10044000780883120313BE007108BF008316A00A48
:100450000319A10AEF298B25831203135708E20021
:10046000AE25F101831203136E08F200720EF0390B
:10047000F039F200F20CF20CF20C720C0F39F200AF
:100480006F08F300730EF039F03972070318F10AA0
:10049000E200AE25F101831203136C08F200720E24
:1004A000F039F039F200F20CF20CF20C720C0F3948
:1004B000F2006D08F300730EF039F039720703187B
:1004C000F10AE200AE25CE3083120313E200AE251E
:1004D000F03083120313E200AE251726E0308316B6
:1004E00003138500F0308600080083120313EC012B
:1004F000ED016D08003C0030031C862A0130031D0D
:10050000862A6C08053C0130031C0301003C0319DA
:10051000D82A5808DF00F1015908F2006C08053CA0
:10052000F4006D08031C013E003CF30074087207E0
:100530000318F10AE00007258312031306140030A4
:100540006D02031DB02A03306C02031DB02A2E3049
:10055000DE00E62483120313EC0A0319ED0A792A5C
:100560004008F8004108F7000A30FA00F901822437
:10057000F1007D08303EF2000318F10A7208831280
:100580000313DE00E624831203134008F800410839
:10059000F7000A30FA00F9019E24F100780883126E
:1005A0000313C0007108C100EC0A0319ED0A792A8F
:1005B000831203135808DF000030F1006D08F107C3
:1005C00059086C070318F10AEC0A0319ED0AE00058
:1005D00007258312031306142C30DE00E624831251
:1005E00003135808DF000030F1006D08F1075908C7
:1005F0006C070318F10AEC0A0319ED0AE00007255D
:100600008312031306144208F8004308F7000A3067
:10061000FA00F9018224F1007D08303EF20003184F
:10062000F10A720883120313DE00E6240800831225
:1006300003134508F1004408DF004708F1004608AD
:10064000E00007258312031306145A08DE00E6248F
:100650000800831203135B0883169B001C141A08FE
:10066000080083120313EA01EB016B08003C003021
:10067000031C422B0130031D422B6A08053C01304C
:10068000031C0301003C03195F2B0030F0006B08D2
:10069000F0075C086A070318F00ADB002923F00062
:1006A00083126B08F1006A08203E840070088313EF
:1006B000800083120313EA0A0319EB0A352B25087D
:1006C000F000700EF039F039F001F000F00CF00C91
:1006D000F00C700C0F39F001F001B0007008B1009F
:1006E0002008F000700EF039F039F001F000F00C45
:1006F000F00CF00C700C0F39F001F900FA01103019
:10070000FB002730FC006024F0007808F100831221
:1007100003132108F200720EF039F039F201F200F1
:10072000F20CF20CF20C720C0F39F201F900FA0122
:10073000E830FB000330FC006024F2007808F10789
:100740000318F20A7208F0077108F100831203130C
:100750002208F200720EF039F039F201F200F20CC8
:10076000F20CF20C720C0F39F201F7006430F80051
:100770007524F2007808F1070318F20A7208F007EE
:100780007108F100831203132308F200720EF0398E
:10079000F039F201F200F20CF20CF20C720C0F398B
:1007A000F201F7000A30F8007524F2007808F1072A
:1007B0000318F20A7208F0077108F100831203139C
:1007C0002408F200720EF039F039F201F200F20C56
:1007D000F20CF20C720C0F39F2017107F1000318E0
:1007E000F00A7108F1007008D50071080800831242
:1007F0000313EC010030F1004B08F10730304A07D9
:100800000318F10AA5000430EC006C08003C031842
:10081000342C4808F8004908F7000A30FA00F901BA
:100820008224F1007D08303EF2000318F10A7208BC
:10083000F100831203136C08203E840071088313B7
:100840008000831203134808F8004908F7000A30B3
:10085000FA00F9019E24F100780883120313C800FE
:100860007108C900EC03052C0030F1004908F107BC
:10087000303048070318F10AA000EC016C08053C71
:10088000031C5F2CF1015D086C070318F10A831645
:100890009B0083126C08203E84008313000883169B
:1008A00003139A001C1555309D00AA309D009C141E
:1008B0009C1C5B2C582C1C118312EC0A3E2C08004B
:1008C000F801F7011030FD00FA0CF90C031C6E2C36
:1008D0007C08F7077B08F8070318F70A0310FB0DDD
:1008E000FC0DFD0B642C770808000930F90077082F
:1008F000F7010310F70CF80C0318F707F90B7A2C23
:1009000077080800FC01FD011030FB00770DFD0D9C
:10091000FC0D7A08FD027908031C790FFC0203180C
:10092000982C7A08FD0779080318790FFC07031043
:10093000F80DF70DFB0B862C7C080800FC01FD016F
:100940001030FB00770DFD0DFC0D7A08FD027908D3
:10095000031C790FFC020318B42C7A08FD077908F0
:100960000318790FFC070310F80DF70DFB0BA22CF1
:100970007708080083120313861106100530FE0065
:100980006F250330831203138500F8240530FE0021
:100990006F250230831203138500F8240530FE0012
:1009A0006F25283083120313DE00E62408308312FB
:1009B0000313DE00E6240C3083120313DE00E6246A
:1009C000063083120313DE00E624080083120313AB
:1009D0005E08F200F20CF20CF20C720C0F3985007A
:1009E000F8245E088500F8242830D4007E2508000D
:1009F0008312031386158611080083120313061051
:100A00000130DE00E6240230FE006F25080083126C
:100A1000031306105F08F1007108013C031D1A2D35
:100A2000F20180308312031360070318F20ADE001C
:100A3000E6242E2D7108023C031D2E2DF2014030BC
:100A40008312031360070318F20AF30072080038D8
:100A5000F20073088038DE00E6242E2D0230FE00FE
:100A60006F25080083120313EA01EB016B08003CB9
:100A70000030031C432D0130031D432D6A080F3C39
:100A80000130031C0301003C03196E2D4D08F100D9
:100A90004C08DF004F08F1006B08F1074E086A07A9
:100AA0000318F10AE000072583120313061400302F
:100AB000F1006B08F10761086A070318F10ADB000F
:100AC0002923013CF1007109013E8312DE00E62476
:100AD00083120313EA0A0319EB0A362D08008E303D
:100AE000FF00000000000000000000000000FF0BFD
:100AF000732D0000FE0B6F2D0000080083120313FE
:100B0000D40CD40C3F30D4050330D4020000D40BF5
:100B1000862D000008008030831603138600013004
:100B20008312E4003A26E3012426E4013A26080071
:100B3000823083160313860001308312E4003A26C4
:100B400044268316A5008312E4013A260130E3000F
:100B50002426803083168600250808008316031398
:100B6000A4010830A200A3012308003C0130031CAB
:100B7000C12D0030031DC12D2208003C0130031897
:100B80000301003C0319E32D2408F100710DFE3927
:100B9000A40083126208013983162404A40083127E
:100BA0006208F100710C7F39E200013083162202E5
:100BB000F2000030031C013E2302F1007208A20083
:100BC0007108A300B42D8030A200A3012308003CCB
:100BD0000130031CF32D0030031DF32D2208003CCF
:100BE000013003180301003C0319152E2408831259
:100BF000E300242683162408F100710C7F39A40039
:100C000001308312E4003A26E4013A2683162208D2
:100C1000F2002308F100710CF20C7F39F100720828
:100C2000F201A2007108A300E62D982508008312A6
:100C30000313E4013A26E30124260130E4003A26B6
:100C40000130E30024260800831203136308F10037
:100C5000710DFE39E3000239E3000030FF39F10085
:100C60000608FD39F20071080038F10072086304CB
:100C700086000800831203136408003C0319422E07
:100C80000615432E061108008312031306080239C5
:100C9000F100710C7F39080083120313EE018230DA
:100CA0008316860008308312EC00ED016D08003CCD
:100CB0000130031C632E0030031D632E6C08003CC2
:100CC000013003180301003C0319802E6E08F00068
:100CD000700DFE39EE000130E4003A2644266E0421
:100CE000EE00E4013A2601306C02F1000030031CF2
:100CF000013E6D02F0007108EC007008ED00562E08
:100D00000130E30024266E0808008312031339081B
:100D1000F1003808C4000B30C6002330DA00172376
:100D20008312031332082E02F2003308031C013E23
:100D30002F02F10072083607F2000318F10A370893
:100D4000F1077208F9007108FA000830FB00FC0195
:100D50006024F1007808831203133007F2000318AF
:100D6000F10A3108F1077208BE007108BF0065087A
:100D7000D700EB21003083123502031DC82E01304D
:100D80003402031DC82E3308EB003208EA00CC2ED3
:100D90002F08EB002E08EA003908F1003808D800C7
:100DA0000330D9006B08C1006A08C0003108C300D5
:100DB0003008C2007522831203136B08C9006A0849
:100DC000C8003108CB003008CA006608DD00F723F0
:100DD0000608F100F10CF10CF10C710C0F390E3C0E
:100DE000031D002F3908F1003808C4000B30C6007D
:100DF0002030DA00172383120313B401B501080071
:100E00000301851B0130013C013003190301F1008E
:100E10000608F200F20CF20CF20C720C0F390D3CC9
:100E20000130031D03017104F1000608F200F20C09
:100E3000F20CF20C720C0F390B3C0130031D030154
:100E40007104003C0319E82E0301051B0130013C2D
:100E5000013003190301F1000608F200F20CF20C54
:100E6000F20C720C0F390D3C0130031D03017104AB
:100E7000003C0319642FBB08031D512FBA08031D42
:100E8000512F00303502031D4D2F01303402031D58
:100E90004D2FB20A0319B30A992FAE0A0319AF0AEC
:100EA000992F83120313B00A0319B10A00303102DB
:100EB000031D632F0A303002031D632FAE0A03198E
:100EC000AF0AB001B101992F83120313BB08031DB0
:100ED0007E2FBA08031D7E2F00303502031D792FA7
:100EE00001303402031D792FB203320A0319B30310
:100EF000992FAE032E0A0319AF03992F8312031300
:100F0000B003300A0319B1033008FF3C03198A2FDC
:100F100000308F2F3108FF3C0130031D0301003CDE
:100F20000319992FAE032E0A0319AF030930B0003D
:100F3000B1019B2FE82E8312031332082E02F20018
:100F40003308031C013E2F02F1007208B93C03195B
:100F5000AB2F0030B02F71080B3C0130031D030193
:100F6000003C0319CD2F00303302031DBB2F00308E
:100F700032020319C72F0330F1003308F107B630EE
:100F800032070318F10AAE007108AF00CB2FB6305C
:100F9000AE000330AF00B001B10132082E02F20002
:100FA0003308031C013E2F02F1007208B53C0319FF
:100FB000DB2F0030E02F7108033C0130031D0301DB
:100FC000003C0319902E00303302031DEB2F00303C
:100FD00032020319F72F0B30F1003308F107B83054
:100FE00032070318F10AAE007108AF00FB2FB830CA
:0E0FF000AE000B30AF00B001B101902E080032
:02400E00503F21
:10420000530079002100210021002100210021001C
:10421000210021002100210021004E0049007B00E7
:1042200055007900210021002100210021002100FA
:10423000210021002100210021004E0049007B00C7
:10424000210032002E004E0049007B002100210099
:10425000210031002F0032002E004E0049007B006B
:1042600050004D00210021002100210021002100EB
:10427000210021002100210021004E0049007B0087
:104280004A00580033004D0047004500210042001D
:104290005500570021002E005300550059002E00F4
:1042A000540058002100530066006D002F002100CB
:1042B00033002F0031002100330031003100350080
:1042D000310030003400380036003000FF00FF00AD
:1042E000300031003200340030003000FF00FF00A9
:1042F000300039003400300030003000FF00FF0093
:00000001FF
